:0A1FE10000010202030304040505D9
:100AE400E4F565F564F563F562C209C206C208C29D
:100AF40007121EA71207317E167F008E0A8F0B7510
:100B0400121675131275081675091C7510167511D1
:100B14005175161675177FEE54E07003020C2B7591
:100B240066007567808E688F69C374A99FFF741609
:100B34009ECF2402CF3400FEE48F618E60F55FF512
:100B44005EF55DF55CF55BF55AAF61AE60AD5FAC2B
:100B54005EAB5DAA5CA95BA85AC3120DEC5026E5F6
:100B640067255DF582E566355CF58374CDF0E55D5A
:100B74002401F55DE4355CF55CE4355BF55BE43557
:100B84005AF55A80C4E4F55DF55CF55BF55AAF613E
:100B9400AE60AD5FAC5EAB5DAA5CA95BA85AC31244
:100BA4000DEC5031AE5CAF5DE5692FF582E5683E32
:100BB400F583E0FDE5672FF582E5663EF583EDF00C
:100BC400EF2401F55DE43EF55CE4355BF55BE4356B
:100BD4005AF55A80B985660A85670B74002480FF2C
:100BE400741634FFFEC3E5139FF513E5129EF51248
:100BF400C3E50D9FF50DE50C9EF50CC3E50F9FF5C0
:100C04000FE50E9EF50EC3E5099FF509E5089EF56F
:100C140008C3E5119FF511E5109EF510C3E5179F74
:100C2400F517E5169EF516D2E843D82090E668E05D
:100C34004409F090E65CE0443DF0D2AF90E680E0F9
:100C440020E105D20A121BF590E680E054F7F05338
:100C54008EF8C20930070512050DC20730092912A2
:100C640015FE5024C209121DC420061690E682E027
:100C740030E704E020E1EF90E682E030E604E02093
:0D0C8400E0E4121C2412206F1211E680C75C
:10050D0090E6B9E070030205BE14700302063B24A9
:10051D00FE70030206BE24FB70030205B8147003BF
:10052D000205B21460731460762405600302071D82
:10053D00122071400302072990E6BBE024FE6022E1
:10054D0014603324FD601114602224067048E50AFE
:10055D0090E6B3F0E50B8037E51290E6B3F0E513C6
:10056D00802DE50C90E6B3F0E50D8023E50E90E6C9
:10057D00B3F0E50F801990E6BAE0FF121C50AA0601
:10058D00A9077B01EA494B600DEE90E6B3F0EF90C1
:10059D00E6B4F0020729020722121F6B0207291287
:1005AD00203D020729121944020729121F5902077B
:1005BD0029122073400302072990E6B8E0247F60DA
:1005CD001514601924027063A206E43325E0FFA21E
:1005DD0008E4334F8041E490E740F0803F90E6BC63
:1005ED00E0547EFF7E00E0D394807C0040047D01CA
:1005FD0080027D00EC4EFEED4F24E1F582741F3E2E
:10060D00F583E493FF3395E0FEEF24A1FFEE34E68E
:10061D008F82F583E0540190E740F0E4A3F090E67B
:10062D008AF090E68B7402F002072902072212204D
:10063D0075400302072990E6B8E024FE60162402F7
:10064D00600302072990E6BAE0B40105C20602076D
:10065D002902072290E6BAE0705590E6BCE0547E80
:10066D00FF7E00E0D394807C0040047D0180027DFC
:10067D0000EC4EFEED4F24E1F582741F3EF583E450
:10068D0093FF3395E0FEEF24A1FFEE34E68F82F564
:10069D0083E054FEF090E6BCE05480131313541F16
:1006AD00FFE0540F2F90E683F0E04420F0806D8042
:1006BD0064122077506690E6B8E024FE601924029B
:1006CD00705A90E6BAE0B40104D206804F90E6BAB3
:1006DD00E064026047803E90E6BCE0547EFF7E0001
:1006ED00E0D394807C0040047D0180027D00EC4EBF
:1006FD00FEED4F24E1F582741F3EF583E493FF3345
:10070D0095E0FEEF24A1FFEE34E68F82F58380089D
:10071D00120080500790E6A0E04401F090E6A0E0C2
:03072D004480F015
:0107300022A6
:0300330002205355
:0420530053D8EF323D
:101EA700758CE0758AC0E58954F04401F589758E13
:081EB70003D28CD2A9D2AF22A4
:03000B000216AB2F
:1016AB00C0E0C0F0C083C082C0D075D000C000C005
:1016BB0001C002C003C004C005C006C007758CE0A2
:1016CB00758AC0D28CE47F607EEAFDFCAB55AA54D0
:1016DB00A953A852C3120DEC5019AF55AE54AD53CC
:1016EB00AC52EF2401F555E43EF554E43DF553E4DB
:1016FB003CF552E47F01FEFDFCAB55AA54A953A85F
:10170B0052C3120DEC7008E5A054F02534F5A0E59A
:10171B002A2401FFE43529FEE4FCFDAB55AA54A9AC
:10172B0053A852C3120DEC700553A0F0C28CD00716
:10173B00D006D005D004D003D002D001D000D0D039
:09174B00D082D083D0F0D0E0324E
:03003B000218DCCC
:1018DC00C0E0C083C082C0D075D000C006C0073045
:1018EC00C041C2C085C114052EE52E7002052DD352
:1018FC00E52E94F4E52D648094814006752D0075D9
:10190C002E00AE2DAF2EEE90F800F0AE2DAF2EEFD8
:10191C00A3F0AE2DAF2E74012FF58274F83EF58333
:10192C00E514F030C105C2C185C114D007D006D072
:08193C00D0D082D083D0E0324C
:030023000219A31C
:1019A300C0E0C083C082C0D075D000C00730983675
:1019B300C298859915052CE52C7002052BD3E52CCF
:1019C300940EE52B648094804006752B00752C00E3
:1019D300AF2C90E7F0EFF0AF2C74F02FF582E434E6
:1019E300E7F583E515F0D007D0D0D082D083D0E0DF
:0119F30032C1
:1016000012010002000000401816118300000102C0
:1016100000010A0600020000004001000902350036
:1016200001010080FA0904000005FF000000070521
:101630000102400000070582020002000705810246
:1016400040000007058602000200070508020002AC
:101650000009022E0001010080FA0904000004FFC5
:10166000000000070501024000000705820240005B
:101670000007050202000200070581024000000485
:1016800003090410035100480059002D0043004392
:101690000044001603490043003800330030003096
:0B16A0000020002000200020000000BF
:10103B0060802800030A030302020307000000027A
:10104B00000002000A2B0B131115111100000000F8
:10105B000000003F020A0303030303070000000222
:10106B00000002000A2B130B1115111100000000D8
:10107B000000003F032D03030303030700000002DE
:10108B00000002000A2B0B131115111100000000B8
:10109B000000003F030A0A0A0A0A0A0700000002BE
:1010AB00000002000A2B130B111511110000000098
:1010BB000000003F602428870000000000000000B3
:1010CB000000000000000000000000000000000015
:1010DB000000000000000000000000004728808096
:0610EB00000011CA4E00D6
:10136C0090E60174CAF090E6F574FFF0902880E0E6
:10137C0090E6F3F0902881E090E6C3F0902882E0AC
:10138C0090E6C1F0902883E090E6C2F0902885E0CA
:10139C0090E6C0F0902886E090E6F4F075AF077404
:1013AC0028F59A7400F59B759DE4E4F59EFF90E694
:1013BC007BE090E67CF00FBF80F490E67174FFF058
:1013CC00F5B490E672E04480F043B680000000E48F
:1013DC0090E6C4F000000090E6C5F0902887E090FD
:1013EC00E6C6F0902888E090E6C7F0902889E09057
:1013FC00E6C8F090288AE090E6C9F090288BE0903F
:10140C00E6CAF090288CE090E6CBF090288DE09026
:0B141C00E6CCF090288EE090E6CDF0CA
:0114270022A2
:03004300021500A3
:0300530002150093
:10150000021EBF00021F1C00021F0600021ED700A1
:10151000021B2300021A37000214FF000220790088
:1015200002207A0002207B00021A740002092800BF
:1015300002207C0002207D000219F400020F3E0010
:1015400002207E000220790002207F00022080001D
:1015500002208100022082000220830002208400F9
:101560000220850002207900022079000220790003
:1015700002208600022087000220880002208900C5
:1015800002208A0002208B0002208C0002208D00A5
:1015900002208E0002208F00022090000220910085
:1015A0000220920002209300022094000220950065
:0815B0000220960002209700C2
:101C240090E682E030E004E020E60B90E682E030CB
:101C3400E119E030E71590E680E04401F07F147E7E
:0C1C4400001215B890E680E054FEF0227B
:101DC40090E682E044C0F090E681F0438701000091
:041DD40000000022E9
:101BF500300A0990E680E0440AF0800790E680E02C
:101C05004408F07FDC7E051215B890E65D74FFF0A0
:0F1C150090E65FF05391EF90E680E054F7F022F5
:021C5000A907E2
:101C5200AE16AF178F828E83A3E064037017AD01B7
:101C620019ED7001228F828E83E07C002FFDEC3E05
:091C7200FEAF0580DF7E007F005B
:011C7B002246
:1015B8008E6E8F6F90E600E054187012E56F24016C
:1015C800FFE4356EC313F56EEF13F56F801590E6E3
:1015D80000E05418FFBF100BE56F25E0F56FE56ECE
:1015E80033F56EE56F156FAE6E7002156E4E6005C1
:0615F800121DD880EE2256
:101DD8007400F58690FDA57C05A3E582458370F91E
:011DE80022D8
:1010F100C18202311040C100014800C105C1040490
:101101004E00000000014500012500043F000000E1
:0A1111000004370000000001350063
:1007310090E600E054E74410F00000000000009053
:10074100E61074A0F000000090E60B7401F090E652
:100751001274E0F0000000E490E613F00000009055
:10076100E61474E2F000000090E61574A0F00000B9
:100771000090E6D27402F090E6047480F00000006C
:100781007402F00000007406F00000007408F0002C
:100791000000E4F000000012136C90E6187408F0F9
:1007A10000000090E619F000000090E61AF0000049
:1007B1000090E61BF0000000E490E671F075B4FFD4
:1007C10090E672F075B67F75B1FF90E670F075B284
:1007D100FF75B5FFC28CD2A053A0FD12204D90E64B
:1007E1001074A0F000000090E611F000000090E607
:1007F1005EE04408F0000000E490E68DF0000000A7
:1008010090E65EE04404F0000000E490E7C0F09060
:10081100E7C4F0A3F0A3F0A3F090E7F0F090E68F27
:100821007440F000000090E65EE04440F0000000FB
:100831007E027F0090F800E4F0A3DFFCDEFA90E690
:10084100987402F0000000E490E699F00000007E48
:10085100027F0090F800E4F0A3DFFCDEFA90E65E90
:10086100E04480F0000000E490E69CF0000000907D
:10087100E69DF00000007F9AFE121FF575270075B6
:1008810028B4754901754A907531107532B8754CA7
:1008910006754D2C12204590E67AE054FEF0E4FDF9
:1008A1007F90121F7D7F647E001215B87DFF7F420D
:1008B100121F7D7F647E001215B87D827F4E121F4C
:1008C1007D7536FF43B101E4F53D90E782E536F0F1
:1008D10090E781E53DF0121EEFE4F52BF52C121D9A
:1008E10027E4F52DF52E12204D1214E07F887E139A
:1008F100121DF71214E07F887E13121DF71214E007
:100901007F887E13121DF7121FC91217547F5512CB
:100911001AB07F887E13121DF7D2F9C2F8E4F545AB
:0609210090E7C0E545F07F
:0109270022AD
:0E1FA100EF2401FBE43EFA7D047F48021E6F30
:10186C00E53DC313FFC374809FF56EE53DD3940033
:10187C0040067536FF43B101E53D700353B1FE7E62
:10188C00297F0B121FA190290CE090E7C1F0902941
:10189C000DE090E7C2F09028EBE536F07A287BEB70
:1018AC007D017F21121E8B9028EB7402F0A37480B3
:1018BC00F07A287BEB7D027F28121E8BE49028EBBC
:1018CC00F0A3E56EF07A287BEB7D027F28021E8B5D
:1011E600E5512401F551E43550F550E4354FF54FFE
:1011F600E4354EF54EE47FE87E03FDFCAB51AA5084
:10120600A94FA84EC3120DEC700F9028EBF07A2868
:101216007BEB7D017F48121E8B7FA07E867D017C45
:1012260000AB51AA50A94FA84EC3120DEC700E1276
:10123600186C90E6907402F0E490E691F07F407EA0
:101246000D7D037C00AB51AA50A94FA84ED3120DB9
:10125600EC400CE4F551F550F54FF54E121E0E30EC
:10126600014075450190E7C0E545F0E5B130E7037B
:101276002005F81212A9C201E4F54590E7C0E5453C
:10128600F01214E07F887E13121DF71214E07F8897
:101296007E13121DF71214E07F887E13121DF712BB
:0312A6001FC9223B
:0215FE00D322F6
:02206F00D3227A
:02207100D32278
:1019440090E680E030E73A00000090E6207402F070
:10195400000000E490E621F000000090E624740208
:10196400F0000000E490E625F000000090E6267404
:1019740002F0000000E490E627F0000000D20280AC
:1019840016000000E490E620F000000090E62174C8
:0F19940040F0000000C20290E6BAE0F546D32210
:101F590090E740E546F0E490E68AF090E68B04F0DD
:021F6900D32281
:08203D0090E6BAE0F526D3227B
:101F6B0090E740E526F0E490E68AF090E68B04F0EB
:021F7B00D3226F
:02207300D32276
:02207500D32274
:02207700D32272
:10008000E4F56AF56B90E6B9E0120E1000B1B3002A
:10009000E9B50266B6029EBB02E5BC038EC103460B
:1000A000C2040CC5042BC60460CA04A1CB00000521
:1000B00009E490E68AF090E68BF090E6A0E020E17B
:1000C000F990E68BE0F56AE4F5B390E60174CAF0C6
:1000D000D20100000090E6047480F0000000740279
:1000E000F0000000E4F002050BE490E68AF090E6F0
:1000F0008BF090E6A0E020E1F990E68BE0F56AD382
:10010000943F4024E4F56B7440256BF582E434E7BA
:10011000F583E0FF74AB256BF582E43428F583EFBB
:10012000F0056BE56BB440DF7F8A7E00121FF5900F
:1001300028ABE0FF7E00121FFE9028ABE0FF7E00A0
:100140001220079028ABE0FF7E001220109028AC10
:10015000E075F004A4FFAEF01220199028ACE07511
:10016000F004A4FFAEF01220229028ACE075F00459
:10017000A4FFAEF012202B9028B0E0C394025013DD
:100180009028CCE090E6C07005744EF08016749C08
:10019000F080119028CCE090E6C07005749FF0804C
:1001A00003749DF09028CEE0F53E9028CBE0F53C1E
:1001B0009028CFE0F5479028D9E0F53BA3E0FEA3D7
:1001C000E07C002400F524EC3EF5239028B1E0F516
:1001D00033E53370037533019028B6E0FEA3E07C6D
:1001E000002400F528EC3EF527A3E0FEA3E0240060
:1001F000F54AEC3EF5499028B2E0FEA3E02400F574
:1002000032EC3EF531A3E0FEA3E02400F54DEC3ED8
:10021000F54C9028BCE0FEA3E02400F544EC3EF54C
:10022000439028BAE0FEA3E02400F530EC3EF52F21
:100230009028E0E0540FF535E4FD7F90121F7D908B
:1002400028ACE0FCA3E0FDA3E0FEA3E0F5428E4174
:100250008D408C3FE542F542E541F541E540F540F2
:10026000E4F53F02050BE4F56B74AB256BF582E416
:100270003428F583E0FF7440256BF582E434E7F51C
:1002800083EFF0056BE56BB440DF000000E490E61F
:100290008AF000000090E68B7440F002050BE490B9
:1002A000E68AF090E68BF090E6A0E020E1F978EBAA
:1002B0007C287D017B017AE679BC7E007F01120DEE
:1002C0006190E6BEE0FF7E0078EC7C287D017B013A
:1002D0007AE77940120D6190E6BAE0C313FF90E629
:1002E000BEE0048059E490E68AF090E68BF090E658
:1002F000A0E020E1F978EB7C287D017B017AE679AA
:10030000BD7E007F01120D6178EC7C287D017B01B0
:100310007AE679BC7E007F01120D6190E6BEE0FFB7
:100320007E0078ED7C287D017B017AE77940120D13
:100330006190E6BAE0C313FF90E6BEE02402FD7AC6
:10034000287BEB02050490E74074EAF0A37403F005
:10035000A3740CF0A37426F0A37407F0A374EEF05A
:10036000A37401F0A37403F0A37453F0300205E406
:10037000A3F0800690E74974FFF0000000E490E6E7
:100380008AF000000090E68B740AF002050BE490FE
:10039000E68AF090E68BF090E6A0E020E1F990E6A6
:1003A0008BE0F56AC298D39400500302050B90E7E6
:1003B00040E0940A5007E02430FF121FAF90E7405E
:1003C000E0B40A057F61121FAF90E740E0B40B056F
:1003D0007F62121FAF90E740E0B40C057F63121FED
:1003E000AF90E740E0B40D057F64121FAF90E74087
:1003F000E0B40E057F65121FAF90E740E0640F6028
:100400000302050B7F66121FAF02050B7AE77B40E4
:100410007D047F48121E6F000000E490E68AF00021
:10042000000090E68B7404F002050BE490E68AF07D
:1004300090E68BF090E6A0E020E1F990E68BE0F505
:100440006AD39401500302050B90E741E0FD7F421F
:10045000121F7D90E740E0FD7F4E121F7D02050BCD
:1004600090E6BCE090290BF07A297B0B7D017F5050
:10047000121E8B7A297B0B7D017F50121E8B90E61A
:10048000BEE0FD7AE77B407F50121E6FE490E68A63
:10049000F000000090E6BEE090E68BF000000080E7
:1004A0006AE490E68AF000000090E68BF00000001D
:1004B00090E6A0E020E1F990E6BCE0D39407404B41
:1004C00078EB7C287D017B017AE679BC7E007F0198
:1004D000120D6190E6BEE0FF7E0078EC7C287D0185
:1004E0007B017AE77940120D6190E6BEE004FD7A67
:1004F000287BEB7F50121E8B90E6BEE004FD7A282D
:0C0500007BEB7F50121E8B8002D322C3C5
:01050C0022CC
:101EBF00C0E0C083C082D2075391EF90E65D7401FA
:081ECF00F0D082D083D0E03294
:101F0600C0E0C083C0825391EF90E65D7404F0D0C8
:061F160082D083D0E0320E
:101F1C00C0E0C083C0825391EF90E65D7402F0D0B4
:061F2C0082D083D0E032F8
:101B2300C0E0C083C08285100C85110D850D8285B0
:101B33000C83A37402F085080E85090F850F828537
:101B43000E83A37407F05391EF90E65D7410F0D009
:061B530082D083D0E032D5
:101ED700C0E0C083C082D2095391EF90E65D7408D9
:081EE700F0D082D083D0E0327C
:101A3700C0E0C083C08290E680E030E72085080CD4
:101A470085090D850D82850C83A37402F085100E20
:101A570085110F850F82850E83A37407F05391EFCD
:0D1A670090E65D7420F0D082D083D0E03294
:0114FF0032BA
:012079003234
:01207A003233
:01207B003232
:101A7400C0E0C083C08290E65EE054FBF00000004A
:101A840090E68F7440F0000000752B00752C0090D8
:101A9400E7F0E4F05391EF90E65FE04404F090E661
:0C1AA4005EE04404F0D082D083D0E03239
:10092800C0E0C0F0C083C082C0D075D000C000C095
:0D09380001C002C003C004C005C006C00716
:1009450090E65EE054F7F090E6A1E020E1F990E74B
:1009550080E0FF120E10097A00098001098F300925
:10096500C3310A07320A45330A76340AA1FE0AABB7
:10097500FF00000AB0752200020AB090E782E0F598
:100985003690E781E0F53D020AB0755600755701CE
:1009950090E68DE0FFC3E5579F7480F86556984053
:1009A50003020AB074802557F582E434E7F583E045
:1009B500FF121FBC0557E55770D6055680D290E744
:1009C50081E07006758DB2020AB090E781E0B4014E
:1009D50006758D64020AB090E781E0B40206758D54
:1009E500D9020AB090E781E0B40306758DE6020AE4
:1009F500B090E781E064046003020AB0758DF302EC
:100A05000AB090E781E070061214E0020AB090E7A0
:100A150081E0B40106121E2F020AB090E781E0B40E
:100A25000206121CD3020AB090E781E0B403051256
:100A35001E50807790E781E0F47070121FC9806BBB
:100A450075560075570190E68DE0FFC3E5579F7415
:100A550080F8655698505474802557F582E434E73C
:100A6500F583E0FF121FAF0557E55770D90556808E
:100A7500D590E781E0F46011E024B0FF121F46E451
:100A8500FF121F467F10121F4690E7817440F07ACF
:100A9500E77B817D217F3C121E8B800F90E781E0F3
:100AA50024FF92058005752200D20300000090E620
:100AB5008DE4F05391EF90E65FE04408F090E65E38
:040AC500E04408F011
:100AC900D007D006D005D004D003D002D001D00081
:0B0AD900D0D0D082D083D0F0D0E0322B
:01207C003231
:01207D003230
:1019F400C0E0C083C08290E65EE054BFF000000007
:101A040090E6987402F000000090E699E4F000007B
:101A140000F52DF52E90F800F0A3F05391EF90E629
:101A24005FE04440F090E65EE04440F0D082D08332
:031A3400D0E032CD
:100F3E00C0E0C0F0C083C082C0D075D000C000C079
:0D0F4E0001C002C003C004C005C006C007FA
:100F5B0090E65EE0547FF090E6A6E020E1F990E6A3
:100F6B009CE0FE90E69DE07C002400F557EC3EF5FE
:100F7B0056E55764054556704D90FC00E0B4EE14F1
:100F8B00A3E0B4440FA3E0B4880AA3E07006A3E087
:100F9B0064336064755800755900C3E5599557E57E
:100FAB00566480F8E558648098504D74002559F5C7
:100FBB008274FC3558F583E0FF121FBC0559E559C7
:100FCB0070D8055880D4755800755900C3E55995EC
:100FDB0057E5566480F8E558648098501B740025DB
:100FEB0059F58274FC3558F583E0FF121FBC055987
:100FFB00E55970D8055880D400000090E69CE4F0C9
:10100B0090E69DF05391EF90E65FE04480F090E620
:05101B005EE04480F0DE
:10102000D007D006D005D004D003D002D001D00024
:0B103000D0D0D082D083D0F0D0E032CE
:01207E00322F
:01207F00322E
:01208000322D
:01208100322C
:01208200322B
:01208300322A
:012084003229
:012085003228
:012086003227
:012087003226
:012088003225
:012089003224
:01208A003223
:01208B003222
:01208C003221
:01208D003220
:01208E00321F
:01208F00321E
:01209000321D
:01209100321C
:01209200321B
:01209300321A
:012094003219
:012095003218
:012096003217
:012097003216
:06111C008F6C8C6D8D6EDE
:10112200536C0753A0BF7F0A7E00121DF7E4F56FD0
:10113200F570C374029570FFE56CA807088002C3BE
:1011420013D8FC30E00543A020800353A0DF7F0AC0
:101152007E00121DF743A0107F0A7E00121DF75376
:10116200A0EF7F0A7E00121DF70570E57070020580
:101172006FC39403E56F6480948040B6E4F56FF525
:1011820070C374099570FFE56EAE6DA807088005FF
:10119200CEC313CE13D8F930E00543A02080035309
:1011A200A0DF7F0A7E00121DF743A0107F0A7E0097
:1011B200121DF753A0EF7F0A7E00121DF70570E59E
:1011C200707002056FC3940AE56F6480948040B129
:1011D20043A0407F0A7E00121DF753A0BF7F0A7E04
:0411E20000021DF7F3
:091FF500AD07AC06E4FF02111C6B
:091FFE00AD07AC067F0402111CC2
:09200700AD07AC067F0502111CB7
:09201000AD07AC067F0602111CAD
:09201900AD07AC067F0102111CA9
:09202200AD07AC067F0202111C9F
:09202B00AD07AC067F0302111C95
:101F7D009028EBEDF0EFC313FF7A287BEB7D010288
:021F8D001E8BA9
:101D4F009028EB7402F0A37480F07A287BEB7D026D
:101D5F007F28121E8BE49028EBF0A3F07A287BEB00
:071D6F007D027F28021E8B9C
:101F4600E49028EBF0A3EFF07A287BEB7D027F3C50
:031F5600021E8BDD
:101F32009028EB7440F0A3EFF07A287BEB7D027FD0
:041F42003C021E8BB4
:101754007FAE121F467F04121F467F10121F467F62
:1017640040121F467FB0121F467F81121F467F80A2
:10177400121F467FA1121F467FA6121F467FA81282
:101784001F467F3F121F467FAD121F467F8B121FDD
:10179400467F30121F467FC8121F467FD3121F4652
:1017A400E4FF121F467FD5121F467F80121F467F1B
:1017B400D9121F467F22121F467FDA121F467F026C
:1017C400121F467F8D121F467F14121F467FDB12A5
:0C17D4001F467F40121F467FAF021F46D9
:021AB0008F6A3B
:101AB200E4FF121F467F10121F46E4F56CE56C240A
:101AC200B6FF121F46E4FF121F467F10121F46E4A4
:101AD200F56BAF6A121F32056BE56BC3946040F27F
:091AE200056CE56CC3940240D4CC
:011AEB0022D8
:0E1DE9007FFC7E08121DF7121FDD7FFC7E08B6
:101DF700EF7803C333CE33CED8F9FFEF4E6007EF4A
:071E07001F70F81E80F52298
:03206300C2822214
:03206600D2822201
:03206900C285220B
:03206C00D28522F8
:06204D0012206602206C67
:101E0E001220637F027E00121DF7122069122066D7
:101E1E007F027E00121DF712206C7F027E00021DD3
:011E2E00F7BC
:101F8F00E4FDFC121E0E0DBD00010CBC0DF5BDF6DF
:011F9F00F24F
:011FA000221E
:0A1FEB00121E2F121FC943B140223D
:0920340053B1BF121E50021FC976
:1014280085423A854139854038853F37E53CB401E6
:1014380002C2A0121FEBE53E60030214CC75220124
:10144800E47FE87E03FDFCAB3AAA39A938A837C384
:10145800120DEC4061E5226401705B7FDD7E0312B2
:1014680015B812186CE53A2418F53AE53934FCF544
:1014780039E53834FFF538E53734FFF537E4FFFE52
:10148800FDE537FC7818120DFD90E7C4EFF0E4FF96
:10149800FEE538FDE4FC7810120DFDA3EFF0E4FF43
:1014A800E539FEE4FDFC7808120DFDA3EFF0E53AFE
:1014B800FFA3EFF0808AE522B40112AE39AF3A12E9
:1014C80015B88009752201E522640160FA122034FA
:0814D800E53CB40102D2A022A0
:101C7C00AD07AC06D3ED9400EC9400401E000000C0
:101C8C00EE90E6D0F0000000ED90E6D1F000000000
:0C1C9C0075BB04000000E5BB30E7FB2234
:081AEC008C6E8D6FAB07AA069A
:101AF400E4FDFCC3ED956FEC956E5022EA90E6D0C0
:101B0400F0000000EB90E6D1F000000075BB05008A
:0E1B14000000E5BB30E7FB0DBD00010C80D5E5
:011B220022A0
:101CFE00AD07AC06000000ED25E0EC3390E6D0F029
:101D0E00000000ED25E090E6D1F000000075BB0468
:091D1E00000000E5BB30E7FB22E8
:1012A900C203121F8F75450290E7C0E545F012147D
:1012B9002875450390E7C0E545F030030302136B39
:1012C900E4F56CF56DC3E56D9528E56C9527500D32
:1012D900121E0E056DE56D70EC056C80E8E53BD3DB
:1012E9009400400CE53BFD7C00AF32AE31121AECA4
:1012F900D3E5249400E52394004007AF24AE2312DC
:101309001CFEE4F56AF56BC3E56B954DE56A954CF2
:10131900502C121CA8E4F56CF56DC3E56D9533747A
:1013290080F8656C98500D121E0E056DE56D70EA1A
:10133900056C80E6056BE56B70CD056A80C9E4F53F
:101349006CF56DC3E56D954AE56C9549500D121E16
:101359000E056DE56D70EC056C80E8AF44AE431287
:021369001C7CEA
:01136B00225F
:101CA800000000E53225E0E5313390E6D0F0000091
:101CB80000E53225E090E6D1F000000075BB040095
:0B1CC8000000E5BB20E7033003F8221A
:101EEF00E490E608F075C83443985053877FD2AC1E
:071EFF0075CBFF75CA6422D8
:0D1FAF00309902C2998F993099FDC2992294
:101D760090000020981CA3AF82AE83E4FCFD7BFAA2
:101D86007AFFF9F8C3120DD65004D2008004C200BF
:061D960080E1C298AF9944
:011D9C002224
:101D2700E490E608F0D28E53897F5389BF43892018
:101D37005389EF438E10758DB243C05043D880C28C
:081D4700C0C2C1D2AED2AF222E
:0D1FBC0030C102C2C18FC130C1FDC2C122BF
:101D9D0090000020C01CA3AF82AE83E4FCFD7BFA53
:101DAD007AFFF9F8C3120DD65004D2008004C20098
:061DBD0080E1C2C0AFC1CD
:011DC30022FD
:0420570075B0092235
:04205B0075B0032237
:04205F0075B0062230
:071FD6007FC47E09121DF714
:041FDD0075B00C22AD
:0D1FC900E4F5B07525FF90E7CBE525F0228B
:1014E000121DF0122057121DF312205B121DF31271
:0F14F000205F121DE9E4F52590E7CBE525F022FA
:101E5000121DF012205F121DF312205B121DF312EF
:0F1E60002057121DE975250390E7CBE525F022E9
:101E2F0012205B7FC47E09121DF7122057121FD696
:101E3F007FC47E09121DF775250190E7CBE525F0CC
:011E4F002270
:101CD3001220577FC47E09121DF712205B7FC47E3A
:101CE30009121DF712205F121FD67FC47E09121D31
:0B1CF300F775250290E7CBE525F022F5
:08204500E4F51DD2E9D2AF223F
:101B590090E678E020E6F9C2E990E678E04480F082
:101B6900EF25E090E679F090E678E030E0F990E64C
:101B790078E04440F090E678E020E6F990E678E0F5
:061B890030E1D6D2E92292
:101BC300A90790E678E020E6F9E51D702390E67812
:101BD300E04480F0E925E090E679F08D18AF03A9A1
:101BE300077519018A1A891BE4F51C751D01D32297
:021BF300C3220B
:101B8F00A90790E678E020E6F9E51D702590E67844
:101B9F00E04480F0E925E0440190E679F08D18AF3C
:101BAF0003A9077519018A1A891BE4F51C751D0312
:041BBF00D322C32248
:03004B00020E366C
:100E3600C0E0C083C082C085C084C086758600C0FD
:100E4600D075D000C000C001C002C003C006C007F4
:100E560090E678E030E206751D06020F2090E678EF
:100E6600E020E10CE51D64026006751D07020F20F7
:100E7600E51D24FE605F14603624FE7003020F1128
:100E860024FC7003020F1D24086003020F20AB1917
:100E9600AA1AA91BAF1C051C8F82758300120D8729
:100EA60090E679F0E51C65187070751D05806B90ED
:100EB600E679E0AB19AA1AA91BAE1C8E82758300CF
:100EC600120DB4751D02E5186401704E90E678E0C7
:100ED6004420F08045E51824FEB51C0790E678E02E
:100EE6004420F0E51814B51C0A90E678E04440F07A
:100EF600751D0090E679E0AB19AA1AA91BAE1C8EE7
:100F060082758300120DB4051C800F90E678E044CC
:100F160040F0751D008003751D005391DFD007D08A
:100F260006D003D002D001D000D0D0D086D084D055
:080F360085D082D083D0E032A7
:101E6F00121B8FE51D24FA600E146006240770F311
:0C1E7F00D322E4F51DD322E4F51DD3228C
:101E8B00121BC3E51D24FA600E146006240770F3C1
:0C1E9B00D322E4F51DD322E4F51DD32270
:030000000217E004
:0C17E000787FE4F6D8FD758170021827B0
:100C9100E709F608DFFA8046E709F208DFFA803E45
:100CA10088828C83E709F0A3DFFA8032E309F60832
:100CB100DFFA8078E309F208DFFA807088828C839A
:100CC100E309F0A3DFFA806489828A83E0A3F6084E
:100CD100DFFA805889828A83E0A3F208DFFA804C28
:100CE10080D280FA80C680D4806980F280338010FF
:100CF10080A680EA809A80A880DA80E280CA803368
:100D010089828A83ECFAE493A3C8C582C8CCC583DF
:100D1100CCF0A3C8C582C8CCC583CCDFE9DEE780AF
:100D21000D89828A83E493A3F608DFF9ECFAA9F02E
:100D3100EDFB2289828A83ECFAE0A3C8C582C8CC84
:100D4100C583CCF0A3C8C582C8CCC583CCDFEADE9D
:100D5100E880DB89828A83E493A3F208DFF980CCFF
:100D610088F0EF60010E4E60C388F0ED2402B404F8
:100D71000050B9F582EB2402B4040050AF2323459F
:060D81008223900CE173D7
:100D8700BB010CE58229F582E5833AF583E0225021
:100D970006E92582F8E622BBFE06E92582F8E2226B
:0D0DA700E58229F582E5833AF583E4932285
:100DB400F8BB010DE58229F582E5833AF583E8F075
:100DC400225006E92582C8F622BBFE05E92582C821
:020DD400F22209
:100DD600EB9FF5F0EA9E42F0E99D42F0EC6480C894
:060DE60064809845F02234
:100DEC00EB9FF5F0EA9E42F0E99D42F0E89C45F05D
:010DFC0022D4
:100DFD00E8600FECC313FCED13FDEE13FEEF13FFD4
:030E0D00D8F122F7
:100E1000D083D082F8E4937012740193700DA3A371
:100E200093F8740193F5828883E473740293686085
:060E3000EFA3A3A380DF85
:1017EC00020AE4E493A3F8E493A34003F68001F225
:1017FC0008DFF48029E493A3F85407240CC8C333FE
:10180C00C4540F4420C8834004F456800146F6DFCC
:10181C00E4800B010204081020408090103BE47E11
:10182C00019360BCA3FF543F30E509541FFEE493C1
:10183C00A360010ECF54C025E060A840B8E493A388
:10184C00FAE493A3F8E493A3C8C582C8CAC583CAB3
:10185C00F0A3C8C582C8CAC583CADFE9DEE780BE6B
:01111B0000D3
:00000001FF
